:020000040000FA
:0400000025EF00F0F8
:0200080034D0F2
:0800180082D0056A046EFF0EA0
:100020000426052200D0D8A01200030E036EE70EAE
:1000300002D8F5D7036AFE0F026EE86A035AD8A009
:1000400012000000020600D0F8D7F86A4F0EAF6E1B
:10005000240EAC6E900EAB6E0001C69A400E926EEE
:10006000E00E936EC00E946E070EB46E0F0EC16E4E
:100070009DD09EAA1BD0060EAB1412E1E1CF3AF040
:10008000E2CF3BF03C2A1EEE80F03C50E126000E11
:10009000E222AECFE7FF3AC0E1FF3BC0E2FF110032
:1000A000AE50AE50AB98AB8811000AD0F2A408D085
:1000B000F294084A092A817A076AD6CF06F011001D
:1000C00011003C503D5C14E03D2AE9CF02F0EACF3C
:1000D00003F00EEE80F03D50E926000EEA22EF50CC
:1000E000026E02C0E9FF03C0EAFFD880120004D00C
:1000F000E868026ED8A0120012003C6A3D6A9D8A30
:100100009F8AF28EF28C12009D9A0EEE80F0000E05
:10011000EE6AE82EFDD73C6A3D6A9D8A1200F29E87
:10012000D8CF5AFEE8CF5BFEE0CF5CFEE9CF5DFEA4
:10013000EACF5EFEE1CF5FFEE2CF60FED9CF61FE87
:10014000DACF62FEF6CF63FEF7CF64FEF5CF65FE31
:10015000F3CF66FEF4CF67FEA6CF68FEF28E0001F5
:10016000A192F29E5ACED8FF5BCEE8FF5CCEE0FFB4
:100170005DCEE9FF5ECEEAFF5FCEE1FF60CEE2FF3B
:1001800061CED9FF62CEDAFF63CEF6FF64CEF7FF11
:1001900065CEF5FF66CEF3FF67CEF4FF68CEA6FF0F
:1001A000F28E10009EA8FED7AD6E120093948A9432
:1001B000929089909292899292948994929689963B
:1001C00092988998929A899A94908B9094928B9213
:1001D00094948B9494968B9694988B98949A8B9AEB
:1001E000939A8A9A226A236A246A256A266A276A67
:1001F000286A296A2A6A2B6A2C6A2D6A2E6A2F6A53
:10020000306A316A326A336A346A356A366A376A02
:10021000386A396A1C6AC5EC0BF0C2EC0DF0939A8F
:100220008A8A320EFADE939A8A9A1A6A1B6A206ABE
:10023000216A63DF69DFCD6AF294F28A870ED56E98
:10024000B16AA192A082D08EA292B00EB16E39DFB7
:100250000A6EBE0E0A5C09E3FE0E0A5C03E3CCEFF5
:1002600004F003D00C6ACCEF04F00AAE22D00C6A82
:100270008D0E0A5C05E10AC00CF00D680E6817D0FF
:100280009D0E0A5C05E10AC00CF00F6810680FD0E3
:10029000AD0E0A5C05E10AC00CF01168126807D0C7
:1002A000BD0E0A5C04E10AC00CF013681468CCEFC0
:1002B00004F00C5204E1CCEF04F0CCEF04F08D0E0E
:1002C0000C5CD8A45DD00D2803E10AC00DF054D019
:1002D000460E0D5C04E11A90899020904CD0470E98
:1002E0000D5C04E11A928992209245D03A0E0D5C81
:1002F00004E11A94899420943ED0490E0D5C04E1E7
:100300001A968996209637D04A0E0D5C04E11A9809
:100310008998209830D04B0E0D5C04E11A9A899A86
:10032000209A29D04C0E0D5C04E11A9C8B90209CE5
:1003300022D04D0E0D5C04E11A9E8B92209E1BD0A4
:100340004E0E0D5C04E11B908B94219014D04F0E47
:100350000D5C04E11B928B9621920DD0500E0D5C2A
:1003600004E11B948B98219406D0510E0D5C03E19F
:100370001B968B9A21960D68CCEF04F0CCEF04F01D
:100380009D0E0C5CD8A4B2EF04F00F2804E10AC063
:100390000FF0B0EF04F00AC010F01052D8A456D0FD
:1003A000460E0F5C04E11A90899020904CD0470EC5
:1003B0000F5C04E11A928992209245D03A0E0F5CAC
:1003C00004E11A94899420943ED0490E0F5C04E114
:1003D0001A968996209637D04A0E0F5C04E11A9837
:1003E0008998209830D04B0E0F5C04E11A9A899AB4
:1003F000209A29D04C0E0F5C04E11A9C8B90209C13
:1004000022D04D0E0F5C04E11A9E8B92209E1BD0D1
:100410004E0E0F5C04E11B908B94219014D04F0E74
:100420000F5C04E11B928B9621920DD0500E0F5C55
:1004300004E11B948B98219406D0510E0F5C03E1CC
:100440001B968B9A21960F68CCEF04F0460E0F5C3A
:1004500034E1225202E12352D8A420801A80D6CF60
:1004600006F0D7CF07F001EEB6F0D8901034E926A9
:10047000000EEA22EECF00F0EFCF01F000C03EF018
:1004800001C03FF03EC000F03FC001F00050062424
:10049000166E01500720176E000E0820186E000E11
:1004A0000920196E18C056F019C057F016C06EF02A
:1004B00017C06FF08980AFEF04F0470E0F5C34E196
:1004C000245202E12552D8A420821A82D6CF06F007
:1004D000D7CF07F002EEB6F0D8901034E926000E20
:1004E000EA22EECF00F0EFCF01F000C040F001C0F3
:1004F00041F040C000F041C001F000500624166EEB
:1005000001500720176E000E0820186E000E0920FB
:10051000196E18C058F019C059F016C070F017C005
:1005200071F08982AFEF04F03A0E0F5C33E126528E
:1005300002E12752D8A420841A84D6CF06F0D7CF60
:1005400007F003EEB6F0D8901034E926000EEA2248
:10055000EECF00F0EFCF01F000C042F001C043F059
:1005600042C000F043C001F000500624166E015056
:100570000720176E000E0820186E000E0920196E55
:1005800018C05AF019C05BF016C072F017C073F0B3
:100590008984E5D1490E0F5C33E1285202E12952EA
:1005A000D8A420861A86D6CF06F0D7CF07F004EE5F
:1005B000B6F0D8901034E926000EEA22EECF00F013
:1005C000EFCF01F000C044F001C045F044C000F09E
:1005D00045C001F000500624166E01500720176E2A
:1005E000000E0820186E000E0920196E18C05CF06D
:1005F00019C05DF016C074F017C075F08986AFD1D0
:100600004A0E0F5C33E12A5202E12B52D8A4208813
:100610001A88D6CF06F0D7CF07F005EEB6F0D890FF
:100620001034E926000EEA22EECF00F0EFCF01F001
:1006300000C046F001C047F046C000F047C001F0DE
:1006400000500624166E01500720176E000E082079
:10065000186E000E0920196E18C05EF019C05FF008
:1006600016C076F017C077F0898879D14B0E0F5CF1
:1006700033E12C5202E12D52D8A4208A1A8AD6CF17
:1006800006F0D7CF07F006EEB6F0D8901034E92682
:10069000000EEA22EECF00F0EFCF01F000C048F0EC
:1006A00001C049F048C000F049C001F000500624E4
:1006B000166E01500720176E000E0820186E000EEF
:1006C0000920196E18C060F019C061F016C078F0EA
:1006D00017C079F0898A43D14C0E0F5C33E12E525A
:1006E00002E12F52D8A4208C1A8CD6CF06F0D7CF97
:1006F00007F007EEB6F0D8901034E926000EEA2293
:10070000EECF00F0EFCF01F000C04AF001C04BF097
:100710004AC000F04BC001F000500624166E015094
:100720000720176E000E0820186E000E0920196EA3
:1007300018C062F019C063F016C07AF017C07BF0E1
:100740008B800DD14D0E0F5C33E1305202E13152FE
:10075000D8A4208E1A8ED6CF06F0D7CF07F008EE99
:10076000B6F0D8901034E926000EEA22EECF00F061
:10077000EFCF01F000C04CF001C04DF04CC000F0D4
:100780004DC001F000500624166E01500720176E70
:10079000000E0820186E000E0920196E18C064F0B3
:1007A00019C065F016C07CF017C07DF08B82D7D0E1
:1007B0004E0E0F5C33E1325202E13352D8A4218055
:1007C0001B80D6CF06F0D7CF07F009EEB6F0D89051
:1007D0001034E926000EEA22EECF00F0EFCF01F050
:1007E00000C04EF001C04FF04EC000F04FC001F00D
:1007F00000500624166E01500720176E000E0820C8
:10080000186E000E0920196E18C066F019C067F046
:1008100016C07EF017C07FF08B84A1D04F0E0F5C06
:1008200033E1345202E13552D8A421821B82D6CF63
:1008300006F0D7CF07F00AEEB6F0D8901034E926CC
:10084000000EEA22EECF00F0EFCF01F000C050F032
:1008500001C051F050C000F051C001F0005006241A
:10086000166E01500720176E000E0820186E000E3D
:100870000920196E18C068F019C069F016C080F020
:1008800017C081F08B866BD0500E0F5C33E136526F
:1008900002E13752D8A421841B84D6CF06F0D7CFEB
:1008A00007F00BEEB6F0D8901034E926000EEA22DD
:1008B000EECF00F0EFCF01F000C052F001C053F0D6
:1008C00052C000F053C001F000500624166E0150D3
:1008D0000720176E000E0820186E000E0920196EF2
:1008E00018C06AF019C06BF016C082F017C083F010
:1008F0008B8835D0510E0F5C32E1385202E139520B
:10090000D8A421861B86D6CF06F0D7CF07F00CEEF1
:10091000B6F0D8901034E926000EEA22EECF00F0AF
:10092000EFCF01F000C054F001C055F054C000F00A
:1009300055C001F000500624166E01500720176EB6
:10094000000E0820186E000E0920196E18C06CF0F9
:1009500019C06DF016C084F017C085F08B8A0F683F
:100960001BD01AD0AD0E0C5C0BE1112803E10AC0BC
:1009700011F004D00AC012F05FEC0AF00DD00CD0D8
:10098000BD0E0C5C09E1132803E10AC013F004D08A
:100990000AC014F050EC0BF01AA03CD056C018F06E
:1009A00057C019F06EC016F06FC017F0D6CF06F022
:1009B000D7CF07F01650065C175007581850085844
:1009C0001950095809501918D8B0800A22E789909F
:1009D0001A9020A01ED0225202E1235219E0D6CF55
:1009E00006F0D7CF07F022500624166E23500720BA
:1009F000176E000E0820186E000E0920196E18C020
:100A000086F019C087F016C09EF017C09FF001D085
:100A1000209037D020A034D086C018F087C019F0BD
:100A20009EC016F09FC017F0D6CF06F0D7CF07F0C4
:100A30001650065C17500758185008581950095896
:100A400009501918D8B0800A1AE71A803EC000F081
:100A50003FC001F000500624166E01500720176EAB
:100A6000000E0820186E000E0920196E18C056F0EE
:100A700019C057F016C06EF017C06FF0898001D012
:100A800089901AA23CD058C018F059C019F070C013
:100A900016F071C017F0D6CF06F0D7CF07F016507A
:100AA000065C175007581850085819500958095033
:100AB0001918D8B0800A22E789921A9220A21ED073
:100AC000245202E1255219E0D6CF06F0D7CF07F025
:100AD00024500624166E25500720176E000E08209D
:100AE000186E000E0920196E18C088F019C089F020
:100AF00016C0A0F017C0A1F001D0209237D020A2DC
:100B000034D088C018F089C019F0A0C016F0A1C078
:100B100017F0D6CF06F0D7CF07F01650065C175067
:100B20000758185008581950095809501918D8B0C2
:100B3000800A1AE71A8240C000F041C001F000505C
:100B40000624166E01500720176E000E0820186E3E
:100B5000000E0920196E18C058F019C059F016C0BF
:100B600070F017C071F0898201D089921AA43CD02C
:100B70005AC018F05BC019F072C016F073C017F0BD
:100B8000D6CF06F0D7CF07F01650065C175007589F
:100B9000185008581950095809501918D8B0800A27
:100BA00022E789941A9420A41ED0265202E12752EB
:100BB00019E0D6CF06F0D7CF07F026500624166EE0
:100BC00027500720176E000E0820186E000E09200F
:100BD000196E18C08AF019C08BF016C0A2F017C0A9
:100BE000A3F001D0209437D020A434D08AC018F0CC
:100BF0008BC019F0A2C016F0A3C017F0D6CF06F034
:100C0000D7CF07F01650065C1750075818500858F1
:100C10001950095809501918D8B0800A1AE71A84CF
:100C200042C000F043C001F000500624166E01508F
:100C30000720176E000E0820186E000E0920196E8E
:100C400018C05AF019C05BF016C072F017C073F0EC
:100C5000898401D089941AA63CD05CC018F05DC08C
:100C600019F074C016F075C017F0D6CF06F0D7CFC4
:100C700007F01650065C17500758185008581950BE
:100C8000095809501918D8B0800A22E789961A968F
:100C900020A61ED0285202E1295219E0D6CF06F034
:100CA000D7CF07F028500624166E29500720176E5C
:100CB000000E0820186E000E0920196E18C08CF066
:100CC00019C08DF016C0A4F017C0A5F001D0209671
:100CD00037D020A634D08CC018F08DC019F0A4C035
:100CE00016F0A5C017F0D6CF06F0D7CF07F01650F4
:100CF000065C1750075818500858195009580950E1
:100D00001918D8B0800A1AE71A8644C000F045C006
:100D100001F000500624166E01500720176E000ED9
:100D20000820186E000E0920196E18C05CF019C05A
:100D30005DF016C074F017C075F0898601D08996F1
:100D40001AA83CD05EC018F05FC019F076C016F04B
:100D500077C017F0D6CF06F0D7CF07F01650065C55
:100D600017500758185008581950095809501918A1
:100D7000D8B0800A22E789981A9820A81ED02A5253
:100D800002E12B5219E0D6CF06F0D7CF07F02A5058
:100D90000624166E2B500720176E000E0820186EC2
:100DA000000E0920196E18C08EF019C08FF016C001
:100DB000A6F017C0A7F001D0209837D020A834D0D3
:100DC0008EC018F08FC019F0A6C016F0A7C017F09B
:100DD000D6CF06F0D7CF07F01650065C175007584D
:100DE000185008581950095809501918D8B0800AD5
:100DF0001AE71A8846C000F047C001F000500624E8
:100E0000166E01500720176E000E0820186E000E97
:100E10000920196E18C05EF019C05FF016C076F098
:100E200017C077F0898801D089981AAA3CD060C091
:100E300018F061C019F078C016F079C017F0D6CF5D
:100E400006F0D7CF07F01650065C17500758185019
:100E500008581950095809501918D8B0800A22E7C3
:100E6000899A1A9A20AA1ED02C5202E12D5219E01A
:100E7000D6CF06F0D7CF07F02C500624166E2D5093
:100E80000720176E000E0820186E000E0920196E3C
:100E900018C090F019C091F016C0A8F017C0A9F0C2
:100EA00001D0209A37D020AA34D090C018F091C039
:100EB00019F0A8C016F0A9C017F0D6CF06F0D7CF0A
:100EC00007F01650065C175007581850085819506C
:100ED000095809501918D8B0800A1AE71A8A48C068
:100EE00000F049C001F000500624166E01500720A2
:100EF000176E000E0820186E000E0920196E18C01B
:100F000060F019C061F016C078F017C079F0898AD6
:100F100001D0899A1AAC3CD062C018F063C019F0B5
:100F20007AC016F07BC017F0D6CF06F0D7CF07F007
:100F30001650065C17500758185008581950095891
:100F400009501918D8B0800A22E78B901A9C20AC5F
:100F50001ED02E5202E12F5219E0D6CF06F0D7CF85
:100F600007F02E500624166E2F500720176E000E25
:100F70000820186E000E0920196E18C092F019C0D2
:100F800093F016C0AAF017C0ABF001D0209C37D068
:100F900020AC34D092C018F093C019F0AAC016F05B
:100FA000ABC017F0D6CF06F0D7CF07F01650065CCF
:100FB000175007581850085819500958095019184F
:100FC000D8B0800A1AE71A8C4AC000F04BC001F072
:100FD00000500624166E01500720176E000E0820E0
:100FE000186E000E0920196E18C062F019C063F067
:100FF00016C07AF017C07BF08B8001D08B901AAEB0
:101000003CD064C018F065C019F07CC016F07DC0FB
:1010100017F0D6CF06F0D7CF07F01650065C175062
:101020000758185008581950095809501918D8B0BD
:10103000800A22E78B921A9E20AE1ED0305202E127
:10104000315219E0D6CF06F0D7CF07F03050062442
:10105000166E31500720176E000E0820186E000E15
:101060000920196E18C094F019C095F016C0ACF0A4
:1010700017C0ADF001D0209E37D020AE34D094C040
:1010800018F095C019F0ACC016F0ADC017F0D6CF6F
:1010900006F0D7CF07F01650065C175007581850C7
:1010A00008581950095809501918D8B0800A1AE779
:1010B0001A8E4CC000F04DC001F000500624166E90
:1010C00001500720176E000E0820186E000E092030
:1010D000196E18C064F019C065F016C07CF017C016
:1010E0007DF08B8201D08B921BA03CD066C018F0A3
:1010F00067C019F07EC016F07FC017F0D6CF06F09B
:10110000D7CF07F01650065C1750075818500858EC
:101110001950095809501918D8B0800A22E78B9441
:101120001B9021A01ED0325202E1335219E0D6CFDB
:1011300006F0D7CF07F032500624166E3350072042
:10114000176E000E0820186E000E0920196E18C0C8
:1011500096F019C097F016C0AEF017C0AFF001D0EE
:10116000219037D021A034D096C018F097C019F044
:10117000AEC016F0AFC017F0D6CF06F0D7CF07F04D
:101180001650065C1750075818500858195009583F
:1011900009501918D8B0800A1AE71B804EC000F019
:1011A0004FC001F000500624166E01500720176E44
:1011B000000E0820186E000E0920196E18C066F087
:1011C00019C067F016C07EF017C07FF08B8401D085
:1011D0008B941BA23CD068C018F069C019F080C085
:1011E00016F081C017F0D6CF06F0D7CF07F0165013
:1011F000065C1750075818500858195009580950DC
:101200001918D8B0800A22E78B961B9221A21ED013
:10121000345202E1355219E0D6CF06F0D7CF07F0AD
:1012200034500624166E35500720176E000E082025
:10123000186E000E0920196E18C098F019C099F0A8
:1012400016C0B0F017C0B1F001D0219237D021A262
:1012500034D098C018F099C019F0B0C016F0B1C0E1
:1012600017F0D6CF06F0D7CF07F01650065C175010
:101270000758185008581950095809501918D8B06B
:10128000800A1AE71B8250C000F051C001F00050E4
:101290000624166E01500720176E000E0820186EE7
:1012A000000E0920196E18C068F019C069F016C048
:1012B00080F017C081F08B8601D08B961BA43CD0A8
:1012C0006AC018F06BC019F082C016F083C017F026
:1012D000D6CF06F0D7CF07F01650065C1750075848
:1012E000185008581950095809501918D8B0800AD0
:1012F00022E78B981B9421A41ED0365202E137526C
:1013000019E0D6CF06F0D7CF07F036500624166E78
:1013100037500720176E000E0820186E000E0920A7
:10132000196E18C09AF019C09BF016C0B2F017C021
:10133000B3F001D0219437D021A434D09AC018F052
:101340009BC019F0B2C016F0B3C017F0D6CF06F0AC
:10135000D7CF07F01650065C17500758185008589A
:101360001950095809501918D8B0800A1AE71B8477
:1013700052C000F053C001F000500624166E015018
:101380000720176E000E0820186E000E0920196E37
:1013900018C06AF019C06BF016C082F017C083F055
:1013A0008B8801D08B981BA63CD06CC018F06DC008
:1013B00019F084C016F085C017F0D6CF06F0D7CF4D
:1013C00007F01650065C1750075818500858195067
:1013D000095809501918D8B0800A22E78B9A1B9631
:1013E00021A61ED0385202E1395219E0D6CF06F0BC
:1013F000D7CF07F038500624166E39500720176EE5
:10140000000E0820186E000E0920196E18C09CF0FE
:1014100019C09DF016C0B4F017C0B5F001D02196E8
:1014200037D021A634D09CC018F09DC019F0B4C0AC
:1014300016F0B5C017F0D6CF06F0D7CF07F016508C
:10144000065C175007581850085819500958095089
:101450001918D8B0800A1AE71B8654C000F055C08E
:1014600001F000500624166E01500720176E000E82
:101470000820186E000E0920196E18C06CF019C0F3
:101480006DF016C084F017C085F08B8A01D08B9A5E
:1014900020501A24006E21501B20016E00100DE117
:1014A000010E095C0AE3086A096A926A896A8B90EC
:1014B0008B928B948B968B988B9A27EF01F0460E2C
:1014C000115C11E112520CE000EEB6F0D89012342B
:1014D000E926000EEA22EECF22F0EFCF23F002D071
:1014E000226A236ADBD0470E115C11E112520CE034
:1014F00000EEB6F0D8901234E926000EEA22EECFC4
:1015000024F0EFCF25F002D0246A256AC7D03A0E26
:10151000115C11E112520CE000EEB6F0D8901234DA
:10152000E926000EEA22EECF26F0EFCF27F002D018
:10153000266A276AB3D0490E115C11E112520CE001
:1015400000EEB6F0D8901234E926000EEA22EECF73
:1015500028F0EFCF29F002D0286A296A9FD04A0EDE
:10156000115C11E112520CE000EEB6F0D89012348A
:10157000E926000EEA22EECF2AF0EFCF2BF002D0C0
:101580002A6A2B6A8BD04B0E115C11E112520CE0CF
:1015900000EEB6F0D8901234E926000EEA22EECF23
:1015A0002CF0EFCF2DF002D02C6A2D6A77D04C0EA4
:1015B000115C11E112520CE000EEB6F0D89012343A
:1015C000E926000EEA22EECF2EF0EFCF2FF002D068
:1015D0002E6A2F6A63D04D0E115C11E112520CE09D
:1015E00000EEB6F0D8901234E926000EEA22EECFD3
:1015F00030F0EFCF31F002D0306A316A4FD04E0E6A
:10160000115C11E112520CE000EEB6F0D8901234E9
:10161000E926000EEA22EECF32F0EFCF33F002D00F
:10162000326A336A3BD04F0E115C11E112520CE06A
:1016300000EEB6F0D8901234E926000EEA22EECF82
:1016400034F0EFCF35F002D0346A356A27D0500E2F
:10165000115C11E112520CE000EEB6F0D890123499
:10166000E926000EEA22EECF36F0EFCF37F002D0B7
:10167000366A376A13D0510E115C10E112520CE039
:1016800000EEB6F0D8901234E926000EEA22EECF32
:1016900038F0EFCF39F002D0386A396A1168120099
:1016A000420E135C07E1145202E11BD802D08A8477
:1016B0001C6804D07B0E135CD8B402D813681200E7
:1016C0001A6A1B6A206A216A89908992899489968C
:1016D0008998899A8B908B928B948B968B988B9A06
:1016E00012001A6A1B6A206A216A8A948990899278
:1016F000899489968998899A8B908B928B948B96F2
:101700008B988B9A226A236A246A256A266A276A3A
:10171000286A296A2A6A2B6A2C6A2D6A2E6A2F6A1D
:10172000306A316A326A336A346A356A366A376ACD
:10173000386A396A1C6A120061EC00F00A6EBE0E4B
:101740000A5C04E3FE0E0A5C01E20C6A0AAE09D0F0
:101750000C6ABD0E0A5C04E10AC00CF01368146840
:1017600013D0BD0E0C5C10E1132803E10AC013F086
:101770000BD00AC014F0145207E0420E135C04E1CF
:101780008A841C6827EF01F0D7D7C30EB86FA20E6A
:10179000B96F990EBA6F980EBB6FC20EBC6F930EE5
:1017A000BD6F120EBE6F8F0EBF6F880EC06F8A0E98
:1017B000C16F230EC26F860EC36FE10EC46F810E20
:1017C000C56FC30EC66F7D0EC76FC50EC86F790E8D
:1017D000C96FE80ECA6F750ECB6F2B0ECC6F720EF1
:1017E000CD6F8B0ECE6F6E0ECF6F0A0ED06F6B0E5D
:1017F000D16FA40ED26F670ED36F5B0ED46F640EE1
:10180000D56F2C0ED66F610ED76F160ED86F5E0E89
:10181000D96F1A0EDA6F5B0EDB6F360EDC6F580E67
:10182000DD6F6A0EDE6F550EDF6FB40EE06F520E85
:10183000E16F150EE26F500EE36F8A0EE46F4D0EEE
:10184000E56F140EE66F4B0EE76FB30EE86F480EB0
:10185000E96F640EEA6F460EEB6F290EEC6F440ED3
:10186000ED6FEE69410EEF6FE70EF06F3F0EF16F17
:10187000E00EF26F3D0EF36FEA0EF46F3B0EF56F64
:10188000030EF66F3A0EF76F2C0EF86F380EF96FE5
:10189000640EFA6F360EFB6FAA0EFC6F340EFD6FEE
:1018A000FE0EFE6F320EFF6F600E0101006F310EF3
:1018B000016FCF0E026F2F0E036F4B0E046F2E0EB3
:1018C000056FD30E066F2C0E076F670E086F2B0E79
:1018D000096F060E0A6F2A0E0B6FB10E0C6F280EE1
:1018E0000D6F660E0E6F270E0F6F260E106F116FA5
:1018F000F10E126F240E136FC50E146F230E156FA9
:10190000A20E166F220E176F890E186F210E196F17
:10191000790E1A6F200E1B6F710E1C6F1F0E1D6F3C
:10192000710E1E6F1E0E1F6F7A0E206F1D0E216F1F
:101930008B0E226F1C0E236FA30E246F1B0E256FC0
:10194000C30E266F1A0E276FE90E286F190E296F26
:10195000170E2A6F190E2B6F4B0E2C6F180E2D6F52
:10196000860E2E6F170E2F6FC70E306F160E316F4B
:101970000E0E326F160E336F5B0E346F150E356F11
:10198000AD0E366F140E376F050E386F140E396FAB
:10199000630E3A6F130E3B6FC50E3C6F120E3D6F18
:1019A0002D0E3E6F120E3F6F990E406F110E416F5C
:1019B0000A0E426F110E436F800E446F100E456F7A
:1019C000FA0E466F0F0E476F780E486F0F0E496F75
:1019D000FA0E4A6F0E0E4B6F810E4C6F0E0E4D6F4E
:1019E0000B0E4E6F0E0E4F6F990E506F0D0E516F06
:1019F0002B0E526F0D0E536FC00E546F0C0E556FA1
:101A0000580E566F0C0E576FF40E586F0B0E596F21
:101A1000930E5A6F0B0E5B6F350E5C6F0B0E5D6F86
:101A2000DA0E5E6F0A0E5F6F820E606F0A0E616FD4
:101A30002C0E626F0A0E636FDA0E646F090E656F0B
:101A40008A0E666F090E676F3C0E686F090E696F2C
:101A5000F10E6A6F080E6B6FA90E6C6F080E6D6F3A
:101A6000620E6E6F080E6F6F1E0E706F080E716F34
:101A7000DC0E726F070E736F9C0E746F070E756F1E
:101A80005F0E766F070E776F230E786F070E796FF4
:101A9000E90E7A6F060E7B6FB10E7C6F060E7D6FBE
:101AA0007A0E7E6F060E7F6F460E806F060E816F78
:101AB000130E826F060E836FE10E846F050E856F25
:101AC000B20E866F050E876F830E886F050E896FC5
:101AD000570E8A6F050E8B6F2B0E8C6F050E8D6F58
:101AE000010E8E6F050E8F6FD90E906F040E916FE1
:101AF000B10E926F040E936F8B0E946F040E956F60
:101B0000660E966F040E976F430E986F040E996FD2
:101B1000200E9A6F040E9B6FFE0E9C6F030E9D6F3E
:101B2000DE0E9E6F030E9F6FBF0EA06F030EA16FA0
:101B3000A00EA26F030EA36F830EA46F030EA56FFA
:101B4000660EA66F030EA76F4B0EA86F030EA96F4C
:101B5000300EAA6F030EAB6F160EAC6F030EAD6F97
:101B6000FD0EAE6F020EAF6FE50EB06F020EB16FDD
:101B7000CD0EB26F020EB36FB60EB46F020EB56F1C
:101B8000000112004C0E0101B86FB96B4F0EBA6F15
:101B9000BB6B510EBC6FBD6B530EBE6FBF6B550E52
:101BA000C06FC16B570EC26FC36B5A0EC46FC56B4B
:101BB0005C0EC66FC76B5E0EC86FC96B600ECA6FD6
:101BC000CB6B620ECC6FCD6B650ECE6FCF6B670E9D
:101BD000D06FD16B690ED26FD36B6B0ED46FD56B98
:101BE0006D0ED66FD76B700ED86FD96B720EDA6F21
:101BF000DB6B740EDC6FDD6B760EDE6FDF6B780EE9
:101C0000E06FE16B7B0EE26FE36B7D0EE46FE56BE3
:101C10007F0EE66FE76B810EE86FE96B840EEA6F6B
:101C2000EB6B860EEC6FED6B880EEE6FEF6B8A0E32
:101C3000F06FF16B8C0EF26FF36B8F0EF46FF56B30
:101C4000910EF66FF76B930EF86FF96B950EFA6FB6
:101C5000FB6B970EFC6FFD6B9A0EFE6FFF6B9C0E7D
:101C60000201006F016B9E0E026F036BA00E046FEA
:101C7000056BA20E066F076BA50E086F096BA70E0A
:101C80000A6F0B6BA90E0C6F0D6BAB0E0E6F0F6B0B
:101C9000AD0E106F116BB00E126F136BB20E146F8E
:101CA000156BB40E166F176BB60E186F196BB80E56
:101CB0001A6F1B6BBB0E1C6F1D6BBD0E1E6F1F6B57
:101CC000BF0E206F216BC10E226F236BC30E246FDA
:101CD000256BC60E266F276BC80E286F296BCA0EA0
:101CE0002A6F2B6BCC0E2C6F2D6BCF0E2E6F2F6BA4
:101CF000D10E306F316BD30E326F336BD50E346F24
:101D0000356BD70E366F376BDA0E386F396BDC0EEA
:101D10003A6F3B6BDE0E3C6F3D6BE00E3E6F3F6BF0
:101D2000E20E406F416BE50E426F436BE70E446F6E
:101D3000456BE90E466F476BEB0E486F496BED0E36
:101D40004A6F4B6BF00E4C6F4D6BF20E4E6F4F6B3C
:101D5000F40E506F516BF60E526F536BF80E546FBA
:101D6000556BFB0E566F576BFD0E586F596B5A69CA
:101D70005B6B010E5C6F5D6F030E5E6F010E5F6F3C
:101D8000060E606F010E616F080E626F010E636FC9
:101D90000A0E646F010E656F0C0E666F010E676FA1
:101DA0000E0E686F010E696F110E6A6F010E6B6F78
:101DB000130E6C6F010E6D6F150E6E6F010E6F6F4F
:101DC000170E706F010E716F190E726F010E736F27
:101DD0001C0E746F010E756F1E0E766F010E776FFD
:101DE000200E786F010E796F220E7A6F010E7B6FD5
:101DF000250E7C6F010E7D6F270E7E6F010E7F6FAB
:101E0000290E806F010E816F2B0E826F010E836F82
:101E10002D0E846F010E856F300E866F010E876F59
:101E2000320E886F010E896F340E8A6F010E8B6F30
:101E3000360E8C6F010E8D6F380E8E6F010E8F6F08
:101E40003B0E906F010E916F3D0E926F010E936FDE
:101E50003F0E946F010E956F410E966F010E976FB6
:101E6000430E986F010E996F460E9A6F010E9B6F8D
:101E7000480E9C6F010E9D6F4A0E9E6F010E9F6F64
:101E80004C0EA06F010EA16F4E0EA26F010EA36F3C
:101E9000510EA46F010EA56F530EA66F010EA76F12
:101EA000550EA86F010EA96F570EAA6F010EAB6FEA
:101EB000590EAC6F010EAD6F5C0EAE6F010EAF6FC1
:101EC0005E0EB06F010EB16F600EB26F010EB36F98
:101ED000620EB46F010EB56F3E0EB86FB96B400E57
:101EE000BA6FBB6B420EBC6FBD6B450EBE6FBF6B56
:101EF000470EC06FC16B490EC26FC36B4C0EC46FEF
:101F0000C56B4E0EC66FC76B500EC86FC96B530EB4
:101F1000CA6FCB6B550ECC6FCD6B570ECE6FCF6BA0
:101F20005A0ED06FD16B5C0ED26FD36B5E0ED46F36
:101F3000D56B600ED66FD76B630ED86FD96B650EFD
:101F4000DA6FDB6B670EDC6FDD6B6A0EDE6FDF6BEB
:101F50006C0EE06FE16B6E0EE26FE36B710EE46F7F
:101F6000E56B730EE66FE76B750EE86FE96B780E45
:101F7000EA6FEB6B7A0EEC6FED6B7C0EEE6FEF6B36
:101F80007F0EF06FF16B810EF26FF36B830EF46FC7
:101F9000F56B860EF66FF76B880EF86FF96B8A0E8D
:101FA000FA6FFB6B8D0EFC6FFD6B8F0EFE6FFF6B80
:101FB000910E0301006F016B940E026F036B960E7E
:101FC000046F056B980E066F076B9B0E086F096B0D
:101FD0009D0E0A6F0B6B9F0E0C6F0D6BA10E0E6F9B
:101FE0000F6BA40E106F116BA60E126F136BA80E61
:101FF000146F156BAB0E166F176BAD0E186F196B58
:10200000AF0E1A6F1B6BB20E1C6F1D6BB40E1E6FE2
:102010001F6BB60E206F216BB90E226F236BBB0EA8
:10202000246F256BBD0E266F276BC00E286F296BA2
:10203000C20E2A6F2B6BC40E2C6F2D6BC70E2E6F2A
:102040002F6BC90E306F316BCB0E326F336BCE0EF0
:10205000346F356BD00E366F376BD20E386F396BED
:10206000D50E3A6F3B6BD70E3C6F3D6BD90E3E6F72
:102070003F6BDC0E406F416BDE0E426F436BE00E38
:10208000446F456BE20E466F476BE50E486F496B38
:10209000E70E4A6F4B6BE90E4C6F4D6BEC0E4E6FBB
:1020A0004F6BEE0E506F516BF00E526F536BF30E81
:1020B000546F556BF50E566F576BF70E586F596B83
:1020C000FA0E5A6F5B6BFC0E5C6F5D6BFE0E5E6F03
:1020D0005F6B010E606F616F030E626F010E636FC5
:1020E000050E646F010E656F080E666F010E676F57
:1020F0000A0E686F010E696F0C0E6A6F010E6B6F2E
:102100000F0E6C6F010E6D6F110E6E6F010E6F6F03
:10211000130E706F010E716F160E726F010E736FDA
:10212000180E746F010E756F1A0E766F010E776FB1
:102130001C0E786F010E796F1F0E7A6F010E7B6F88
:10214000210E7C6F010E7D6F230E7E6F010E7F6F5F
:10215000260E806F010E816F280E826F010E836F35
:102160002A0E846F010E856F2D0E866F010E876F0C
:102170002F0E886F010E896F310E8A6F010E8B6FE3
:10218000340E8C6F010E8D6F360E8E6F010E8F6FB9
:10219000380E906F010E916F3B0E926F010E936F90
:1021A0003D0E946F010E956F3F0E966F010E976F67
:1021B000420E986F010E996F440E9A6F010E9B6F3D
:1021C000460E9C6F010E9D6F490E9E6F010E9F6F14
:1021D0004B0EA06F010EA16F4D0EA26F010EA36FEB
:1021E000500EA46F010EA56F520EA66F010EA76FC1
:1021F000540EA86F010EA96F570EAA6F010EAB6F98
:10220000590EAC6F010EAD6F5B0EAE6F010EAF6F6E
:102210005D0EB06F010EB16F600EB26F010EB36F45
:10222000620EB46F010EB56F470E0501B86FB96B42
:102230004A0EBA6FBB6B4C0EBC6FBD6B4E0EBE6FC1
:10224000BF6B500EC06FC16B530EC26FC36B550E88
:10225000C46FC56B570EC66FC76B590EC86FC96B7D
:102260005C0ECA6FCB6B5E0ECC6FCD6B600ECE6F0B
:10227000CF6B620ED06FD16B650ED26FD36B670ED2
:10228000D46FD56B690ED66FD76B6B0ED86FD96BC9
:102290006E0EDA6FDB6B700EDC6FDD6B720EDE6F55
:1022A000DF6B740EE06FE16B770EE26FE36B790E1C
:1022B000E46FE56B7B0EE66FE76B7D0EE86FE96B15
:1022C000800EEA6FEB6B820EEC6FED6B840EEE6F9F
:1022D000EF6B860EF06FF16B890EF26FF36B8B0E66
:1022E000F46FF56B8D0EF66FF76B8F0EF86FF96B61
:1022F000920EFA6FFB6B940EFC6FFD6B960EFE6FE9
:10230000FF6B980E0601006F016B9B0E026F036B53
:102310009D0E046F056B9F0E066F076BA10E086F75
:10232000096BA30E0A6F0B6BA60E0C6F0D6BA80E3C
:102330000E6F0F6BAA0E106F116BAC0E126F136B3A
:10234000AF0E146F156BB10E166F176BB30E186FBF
:10235000196BB50E1A6F1B6BB80E1C6F1D6BBA0E86
:102360001E6F1F6BBC0E206F216BBE0E226F236B86
:10237000C10E246F256BC30E266F276BC50E286F09
:10238000296BC70E2A6F2B6BCA0E2C6F2D6BCC0ED0
:102390002E6F2F6BCE0E306F316BD00E326F336BD2
:1023A000D30E346F356BD50E366F376BD70E386F53
:1023B000396BD90E3A6F3B6BDC0E3C6F3D6BDE0E1A
:1023C0003E6F3F6BE00E406F416BE20E426F436B1E
:1023D000E50E446F456BE70E466F476BE90E486F9D
:1023E000496BEB0E4A6F4B6BEE0E4C6F4D6BF00E64
:1023F0004E6F4F6BF20E506F516BF40E526F536B6A
:10240000F70E546F556BF90E566F576BFB0E586FE6
:10241000596BFD0E5A6F5B6B5C695D6B020E5E6FF4
:10242000010E5F6F040E606F010E616F060E626F2A
:10243000010E636F080E646F010E656F0B0E666F01
:10244000010E676F0D0E686F010E696F0F0E6A6FD8
:10245000010E6B6F110E6C6F010E6D6F140E6E6FAF
:10246000010E6F6F160E706F010E716F180E726F86
:10247000010E736F1A0E746F010E756F1D0E766F5D
:10248000010E776F1F0E786F010E796F210E7A6F34
:10249000010E7B6F230E7C6F010E7D6F260E7E6F0B
:1024A000010E7F6F280E806F010E816F2A0E826FE2
:1024B000010E836F2C0E846F010E856F2F0E866FB9
:1024C000010E876F310E886F010E896F330E8A6F90
:1024D000010E8B6F350E8C6F010E8D6F380E8E6F67
:1024E000010E8F6F3A0E906F010E916F3C0E926F3E
:1024F000010E936F3E0E946F010E956F410E966F15
:10250000010E976F430E986F010E996F450E9A6FEB
:10251000010E9B6F470E9C6F010E9D6F4A0E9E6FC2
:10252000010E9F6F4C0EA06F010EA16F4E0EA26F99
:10253000010EA36F500EA46F010EA56F530EA66F70
:10254000010EA76F550EA86F010EA96F570EAA6F47
:10255000010EAB6F590EAC6F010EAD6F5B0EAE6F1F
:10256000010EAF6F5E0EB06F010EB16F600EB26FF5
:10257000010EB36F620EB46F010EB56F470EB86FE8
:10258000B96B4A0EBA6FBB6B4C0EBC6FBD6B4E0E77
:10259000BE6FBF6B500EC06FC16B520EC26FC36B6C
:1025A000540EC46FC56B560EC66FC76B580EC86FFE
:1025B000C96B5A0ECA6FCB6B5C0ECC6FCD6B5E0EC7
:1025C000CE6FCF6B610ED06FD16B630ED26FD36BBA
:1025D000650ED46FD56B670ED66FD76B690ED86F4B
:1025E000D96B6B0EDA6FDB6B6D0EDC6FDD6B6F0E14
:1025F000DE6FDF6B710EE06FE16B730EE26FE36B0A
:10260000750EE46FE56B780EE66FE76B7A0EE86F98
:10261000E96B7C0EEA6FEB6B7E0EEC6FED6B800E60
:10262000EE6FEF6B820EF06FF16B840EF26FF36B57
:10263000860EF46FF56B880EF66FF76B8A0EF86FE7
:10264000F96B8C0EFA6FFB6B8F0EFC6FFD6B910EAE
:10265000FE6FFF6B930E0701006F016B950E026F0B
:10266000036B970E046F056B990E066F076B9B0E3D
:10267000086F096B9D0E0A6F0B6B9F0E0C6F0D6B35
:10268000A10E0E6F0F6BA30E106F116BA50E126FC4
:10269000136BA80E146F156BAA0E166F176BAC0E8A
:1026A000186F196BAE0E1A6F1B6BB00E1C6F1D6B83
:1026B000B20E1E6F1F6BB40E206F216BB60E226F11
:1026C000236BB80E246F256BBA0E266F276BBC0EDA
:1026D000286F296BBF0E2A6F2B6BC10E2C6F2D6BD1
:1026E000C30E2E6F2F6BC50E306F316BC70E326F5E
:1026F000336BC90E346F356BCB0E366F376BCD0E27
:10270000386F396BCF0E3A6F3B6BD10E3C6F3D6B20
:10271000D30E3E6F3F6BD60E406F416BD80E426FAB
:10272000436BDA0E446F456BDC0E466F476BDE0E73
:10273000486F496BE00E4A6F4B6BE20E4C6F4D6B6E
:10274000E40E4E6F4F6BE60E506F516BE80E526FFA
:10275000536BEA0E546F556BED0E566F576BEF0EC1
:10276000586F596BF10E5A6F5B6BF30E5C6F5D6BBC
:10277000F50E5E6F5F6BF70E606F616BF90E626F47
:10278000636BFB0E646F656BFD0E666F676B68694C
:10279000696B010E6A6F6B6F040E6C6F010E6D6FCB
:1027A000060E6E6F010E6F6F080E706F010E716F67
:1027B0000A0E726F010E736F0C0E746F010E756F3F
:1027C0000E0E766F010E776F100E786F010E796F17
:1027D000120E7A6F010E7B6F140E7C6F010E7D6FEF
:1027E000160E7E6F010E7F6F180E806F010E816FC7
:1027F0001A0E826F010E836F1D0E846F010E856F9E
:102800001F0E866F010E876F210E886F010E896F74
:10281000230E8A6F010E8B6F250E8C6F010E8D6F4C
:10282000270E8E6F010E8F6F290E906F010E916F24
:102830002B0E926F010E936F2D0E946F010E956FFC
:102840002F0E966F010E976F310E986F010E996FD4
:10285000340E9A6F010E9B6F360E9C6F010E9D6FAA
:10286000380E9E6F010E9F6F3A0EA06F010EA16F82
:102870003C0EA26F010EA36F3E0EA46F010EA56F5A
:10288000400EA66F010EA76F420EA86F010EA96F32
:10289000440EAA6F010EAB6F460EAC6F010EAD6F0A
:1028A000480EAE6F010EAF6F4B0EB06F010EB16FE1
:1028B0004D0EB26F010EB36F4F0EB46F010EB56FB8
:1028C000910EB86FB96B920EBA6FBB6B940EBC6F62
:1028D000BD6B950EBE6FBF6B960EC06FC16B980E31
:1028E000C26FC36B990EC46FC56B9A0EC66FC76B70
:1028F0009B0EC86FC96B9D0ECA6FCB6B9E0ECC6FC3
:10290000CD6B9F0ECE6FCF6BA10ED06FD16BA20E91
:10291000D26FD36BA30ED46FD56BA40ED66FD76BCB
:10292000A60ED86FD96BA70EDA6FDB6BA80EDC6F23
:10293000DD6BA90EDE6FDF6BAB0EE06FE16BAC0EF3
:10294000E26FE36BAD0EE46FE56BAF0EE66FE76B26
:10295000B00EE86FE96BB10EEA6FEB6BB20EEC6F85
:10296000ED6BB40EEE6FEF6BB50EF06FF16BB60E54
:10297000F26FF36BB70EF46FF56BB90EF66FF76B82
:10298000BA0EF86FF96BBB0EFA6FFB6BBD0EFC6FE6
:10299000FD6BBE0EFE6FFF6BBF0E0801006F016B7B
:1029A000C00E026F036BC20E046F056BC30E066F81
:1029B000076BC40E086F096BC60E0A6F0B6BC70E50
:1029C0000C6F0D6BC80E0E6F0F6BC90E106F116B75
:1029D000CB0E126F136BCC0E146F156BCD0E166FE2
:1029E000176BCE0E186F196BD00E1A6F1B6BD10EB2
:1029F0001C6F1D6BD20E1E6F1F6BD40E206F216BD0
:102A0000D50E226F236BD60E246F256BD70E266F43
:102A1000276BD90E286F296BDA0E2A6F2B6BDB0E12
:102A20002C6F2D6BDD0E2E6F2F6BDE0E306F316B2A
:102A3000DF0E326F336BE00E346F356BE20E366FA4
:102A4000376BE30E386F396BE40E3A6F3B6BE50E74
:102A50003C6F3D6BE70E3E6F3F6BE80E406F416B86
:102A6000E90E426F436BEB0E446F456BEC0E466F05
:102A7000476BED0E486F496BEE0E4A6F4B6BF00ED5
:102A80004C6F4D6BF10E4E6F4F6BF20E506F516BE2
:102A9000F30E526F536BF50E546F556BF60E566F67
:102AA000576BF70E586F596BF90E5A6F5B6BFA0E36
:102AB0005C6F5D6BFB0E5E6F5F6BFC0E606F616B3E
:102AC000FE0E626F636B6469656B666B010E676F08
:102AD000020E686F010E696F030E6A6F010E6B6F55
:102AE000040E6C6F010E6D6F050E6E6F010E6F6F31
:102AF000070E706F010E716F080E726F010E736F0B
:102B0000090E746F010E756F0A0E766F010E776FE6
:102B10000C0E786F010E796F0D0E7A6F010E7B6FC0
:102B20000E0E7C6F010E7D6F100E7E6F010E7F6F9B
:102B3000110E806F010E816F120E826F010E836F76
:102B4000130E846F010E856F150E866F010E876F51
:102B5000160E886F010E896F170E8A6F010E8B6F2C
:102B6000190E8C6F010E8D6F1A0E8E6F010E8F6F06
:102B70001B0E906F010E916F1C0E926F010E936FE2
:102B80001E0E946F010E956F1F0E966F010E976FBC
:102B9000200E986F010E996F210E9A6F010E9B6F98
:102BA000230E9C6F010E9D6F240E9E6F010E9F6F72
:102BB000250EA06F010EA16F270EA26F010EA36F4D
:102BC000280EA46F010EA56F290EA66F010EA76F28
:102BD0002A0EA86F010EA96F2C0EAA6F010EAB6F03
:102BE0002D0EAC6F010EAD6F2E0EAE6F010EAF6FDE
:102BF0002F0EB06F010EB16F310EB26F010EB36FB9
:102C0000320EB46F010EB56FA50EB86FB96BA60E7C
:102C1000BA6FBB6BA80EBC6FBD6BA90EBE6FBF6B4E
:102C2000AB0EC06FC16BAC0EC26FC36BAE0EC46F88
:102C3000C56BAF0EC66FC76BB10EC86FC96BB20E56
:102C4000CA6FCB6BB40ECC6FCD6BB50ECE6FCF6BA6
:102C5000B70ED06FD16BB80ED26FD36BBA0ED46FE4
:102C6000D56BBB0ED66FD76BBD0ED86FD96BBE0EB2
:102C7000DA6FDB6BC00EDC6FDD6BC20EDE6FDF6BFD
:102C8000C30EE06FE16BC50EE26FE36BC60EE46F3F
:102C9000E56BC80EE66FE76BC90EE86FE96BCB0E0C
:102CA000EA6FEB6BCC0EEC6FED6BCE0EEE6FEF6B55
:102CB000CF0EF06FF16BD10EF26FF36BD20EF46F9B
:102CC000F56BD40EF66FF76BD50EF86FF96BD70E68
:102CD000FA6FFB6BD80EFC6FFD6BDA0EFE6FFF6BAD
:102CE000DB0E0901006F016BDD0E026F036BDE0E60
:102CF000046F056BE00E066F076BE10E086F096B42
:102D0000E30E0A6F0B6BE40E0C6F0D6BE60E0E6F8D
:102D10000F6BE70E106F116BE90E126F136BEA0E5B
:102D2000146F156BEC0E166F176BED0E186F196B99
:102D3000EF0E1A6F1B6BF00E1C6F1D6BF20E1E6FE9
:102D40001F6BF30E206F216BF50E226F236BF60EB7
:102D5000246F256BF80E266F276BF90E286F296BF1
:102D6000FB0E2A6F2B6BFC0E2C6F2D6BFE0E2E6F45
:102D70002F6B3069316B010E326F336F020E346F7F
:102D8000010E356F040E366F010E376F050E386F6A
:102D9000010E396F070E3A6F010E3B6F080E3C6F44
:102DA000010E3D6F0A0E3E6F010E3F6F0B0E406F1E
:102DB000010E416F0D0E426F010E436F0E0E446FF8
:102DC000010E456F100E466F010E476F110E486FD2
:102DD000010E496F130E4A6F010E4B6F140E4C6FAC
:102DE000010E4D6F160E4E6F010E4F6F180E506F85
:102DF000010E516F190E526F010E536F1B0E546F5F
:102E0000010E556F1C0E566F010E576F1E0E586F38
:102E1000010E596F1F0E5A6F010E5B6F210E5C6F12
:102E2000010E5D6F220E5E6F010E5F6F240E606FEC
:102E3000010E616F250E626F010E636F270E646FC6
:102E4000010E656F280E666F010E676F2A0E686FA0
:102E5000010E696F2B0E6A6F010E6B6F2D0E6C6F7A
:102E6000010E6D6F2E0E6E6F010E6F6F300E706F54
:102E7000010E716F310E726F010E736F330E746F2E
:102E8000010E756F340E766F010E776F360E786F08
:102E9000010E796F370E7A6F010E7B6F390E7C6FE2
:102EA000010E7D6F3A0E7E6F010E7F6F3C0E806FBC
:102EB000010E816F3D0E826F010E836F3F0E846F96
:102EC000010E856F400E866F010E876F420E886F70
:102ED000010E896F430E8A6F010E8B6F450E8C6F4A
:102EE000010E8D6F460E8E6F010E8F6F480E906F24
:102EF000010E916F490E926F010E936F4B0E946FFE
:102F0000010E956F4C0E966F010E976F4E0E986FD7
:102F1000010E996F4F0E9A6F010E9B6F510E9C6FB1
:102F2000010E9D6F520E9E6F010E9F6F540EA06F8B
:102F3000010EA16F550EA26F010EA36F570EA46F65
:102F4000010EA56F580EA66F010EA76F5A0EA86F3F
:102F5000010EA96F5B0EAA6F010EAB6F5D0EAC6F19
:102F6000010EAD6F5E0EAE6F010EAF6F600EB06FF3
:102F7000010EB16F610EB26F010EB36F630EB46FCD
:102F8000010EB56F5B0EB86FB96B5D0EBA6FBB6BA0
:102F90005F0EBC6FBD6B600EBE6FBF6B620EC06F0D
:102FA000C16B640EC26FC36B660EC46FC56B670ED8
:102FB000C66FC76B690EC86FC96B6B0ECA6FCB6BE0
:102FC0006D0ECC6FCD6B6E0ECE6FCF6B700ED06F63
:102FD000D16B720ED26FD36B740ED46FD56B750E2E
:102FE000D66FD76B770ED86FD96B790EDA6FDB6B34
:102FF0007A0EDC6FDD6B7C0EDE6FDF6B7E0EE06FBA
:10300000E16B800EE26FE36B810EE46FE56B830E84
:10301000E66FE76B850EE86FE96B870EEA6FEB6B87
:10302000880EEC6FED6B8A0EEE6FEF6B8C0EF06F0F
:10303000F16B8E0EF26FF36B8F0EF46FF56B910EDA
:10304000F66FF76B930EF86FF96B950EFA6FFB6BDB
:10305000960EFC6FFD6B980EFE6FFF6B9A0E0A01C9
:10306000006F016B9C0E026F036B9D0E046F056B6E
:103070009F0E066F076BA10E086F096BA30E0A6FF8
:103080000B6BA40E0C6F0D6BA60E0E6F0F6BA80EC4
:10309000106F116BA90E126F136BAB0E146F156BC3
:1030A000AD0E166F176BAF0E186F196BB00E1A6F4F
:1030B0001B6BB20E1C6F1D6BB40E1E6F1F6BB60E1A
:1030C000206F216BB70E226F236BB90E246F256B17
:1030D000BB0E266F276BBD0E286F296BBE0E2A6FA5
:1030E0002B6BC00E2C6F2D6BC20E2E6F2F6BC40E70
:1030F000306F316BC50E326F336BC70E346F356B6B
:10310000C90E366F376BCB0E386F396BCC0E3A6FFA
:103110003B6BCE0E3C6F3D6BD00E3E6F3F6BD20EC5
:10312000406F416BD30E426F436BD50E446F456BBE
:10313000D70E466F476BD80E486F496BDA0E4A6F51
:103140004B6BDC0E4C6F4D6BDE0E4E6F4F6BDF0E1C
:10315000506F516BE10E526F536BE30E546F556B12
:10316000E50E566F576BE60E586F596BE80E5A6FA7
:103170005B6BEA0E5C6F5D6BEC0E5E6F5F6BED0E72
:10318000606F616BEF0E626F636BF10E646F656B66
:10319000F30E666F676BF40E686F696BF60E6A6FFD
:1031A0006B6BF80E6C6F6D6BFA0E6E6F6F6BFB0EC8
:1031B000706F716BFD0E726F736B7469756B010EBE
:1031C000766F776F020E786F010E796F040E7A6F4B
:1031D000010E7B6F060E7C6F010E7D6F070E7E6FFA
:1031E000010E7F6F090E806F010E816F0B0E826FD3
:1031F000010E836F0D0E846F010E856F0E0E866FAC
:10320000010E876F100E886F010E896F120E8A6F84
:10321000010E8B6F140E8C6F010E8D6F150E8E6F5D
:10322000010E8F6F170E906F010E916F190E926F36
:10323000010E936F1B0E946F010E956F1C0E966F0F
:10324000010E976F1E0E986F010E996F200E9A6FE8
:10325000010E9B6F220E9C6F010E9D6F230E9E6FC1
:10326000010E9F6F250EA06F010EA16F270EA26F9A
:10327000010EA36F290EA46F010EA56F2A0EA66F73
:10328000010EA76F2C0EA86F010EA96F2E0EAA6F4C
:10329000010EAB6F300EAC6F010EAD6F310EAE6F25
:1032A000010EAF6F330EB06F010EB16F350EB26FFE
:1032B000010EB36F360EB46F010EB56F430EB86FCB
:1032C000B96B440EBA6FBB6B460EBC6FBD6B470E3D
:1032D000BE6FBF6B490EC06FC16B4A0EC26FC36B2E
:1032E0004C0EC46FC56B4D0EC66FC76B4F0EC86FCB
:1032F000C96B500ECA6FCB6B520ECC6FCD6B540E98
:10330000CE6FCF6B550ED06FD16B570ED26FD36B84
:10331000580ED46FD56B5A0ED66FD76B5B0ED86F25
:10332000D96B5D0EDA6FDB6B5E0EDC6FDD6B600EF2
:10333000DE6FDF6B620EE06FE16B630EE26FE36BDB
:10334000650EE46FE56B660EE66FE76B680EE86F7F
:10335000E96B690EEA6FEB6B6B0EEC6FED6B6C0E4D
:10336000EE6FEF6B6E0EF06FF16B6F0EF26FF36B33
:10337000710EF46FF56B730EF66FF76B740EF86FDA
:10338000F96B760EFA6FFB6B770EFC6FFD6B790EA7
:10339000FE6FFF6B7A0E0B01006F016B7C0E026FEC
:1033A000036B7D0E046F056B7F0E066F076B800E3F
:1033B000086F096B820E0A6F0B6B840E0C6F0D6B1E
:1033C000850E0E6F0F6B870E106F116B880E126FCC
:1033D000136B8A0E146F156B8B0E166F176B8D0E99
:1033E000186F196B8E0E1A6F1B6B900E1C6F1D6B76
:1033F000910E1E6F1F6B930E206F216B950E226F27
:10340000236B960E246F256B980E266F276B990EF3
:10341000286F296B9B0E2A6F2B6B9C0E2C6F2D6BCC
:103420009E0E2E6F2F6B9F0E306F316BA10E326F81
:10343000336BA30E346F356BA40E366F376BA60E4D
:10344000386F396BA70E3A6F3B6BA90E3C6F3D6B23
:10345000AA0E3E6F3F6BAC0E406F416BAD0E426FDC
:10346000436BAF0E446F456BB00E466F476BB20EA9
:10347000486F496BB40E4A6F4B6BB50E4C6F4D6B7A
:10348000B70E4E6F4F6BB80E506F516BBA0E526F36
:10349000536BBB0E546F556BBD0E566F576BBE0E04
:1034A000586F596BC00E5A6F5B6BC10E5C6F5D6BD2
:1034B000C30E5E6F5F6BC50E606F616BC60E626F91
:1034C000636BC80E646F656BC90E666F676BCB0E5E
:1034D000686F696BCC0E6A6F6B6BCE0E6C6F6D6B29
:1034E000CF0E6E6F6F6BD10E706F716BD20E726FED
:1034F000736BD40E746F756BD60E766F776BD70EB9
:10350000786F796BD90E7A6F7B6BDA0E7C6F7D6B7F
:10351000DC0E7E6F7F6BDD0E806F816BDF0E826F46
:10352000836BE00E846F856BE20E866F876BE40E13
:10353000886F896BE50E8A6F8B6BE70E8C6F8D6BD6
:10354000E80E8E6F8F6BEA0E906F916BEB0E926FA1
:10355000936BED0E946F956BEE0E966F976BF00E6E
:10356000986F996BF10E9A6F9B6BF30E9C6F9D6B2E
:10357000F50E9E6F9F6BF60EA06FA16BF80EA26FFB
:10358000A36BF90EA46FA56BFB0EA66FA76BFC0EC9
:10359000A86FA96BFE0EAA6FAB6BAC69AD6B010E89
:1035A000AE6FAF6F020EB06F010EB16F040EB26F4F
:1035B000010EB36F060EB46F010EB56F960EB86FA5
:1035C000B96B970EBA6FBB6B990EBC6FBD6B9A0E41
:1035D000BE6FBF6B9B0EC06FC16B9C0EC26FC36B87
:1035E0009E0EC46FC56B9F0EC66FC76BA00EC86FD3
:1035F000C96BA20ECA6FCB6BA30ECC6FCD6BA40EA2
:10360000CE6FCF6BA50ED06FD16BA70ED26FD36BE1
:10361000A80ED46FD56BA90ED66FD76BAB0ED86F33
:10362000D96BAC0EDA6FDB6BAD0EDC6FDD6BAE0E03
:10363000DE6FDF6BB00EE06FE16BB10EE26FE36B3C
:10364000B20EE46FE56BB30EE66FE76BB50EE86F95
:10365000E96BB60EEA6FEB6BB70EEC6FED6BB90E64
:10366000EE6FEF6BBA0EF06FF16BBB0EF26FF36B98
:10367000BC0EF46FF56BBE0EF66FF76BBF0EF86FF6
:10368000F96BC00EFA6FFB6BC20EFC6FFD6BC30EC5
:10369000FE6FFF6BC40E0C01006F016BC50E026F55
:1036A000036BC70E046F056BC80E066F076BC90E60
:1036B000086F096BCA0E0A6F0B6BCC0E0C6F0D6B8B
:1036C000CD0E0E6F0F6BCE0E106F116BD00E126FF2
:1036D000136BD10E146F156BD20E166F176BD30EC2
:1036E000186F196BD50E1A6F1B6BD60E1C6F1D6BE6
:1036F000D70E1E6F1F6BD80E206F216BDA0E226F54
:10370000236BDB0E246F256BDC0E266F276BDE0E22
:10371000286F296BDF0E2A6F2B6BE00E2C6F2D6B41
:10372000E10E2E6F2F6BE30E306F316BE40E326FB4
:10373000336BE50E346F356BE70E366F376BE80E83
:10374000386F396BE90E3A6F3B6BEA0E3C6F3D6B9D
:10375000EC0E3E6F3F6BED0E406F416BEE0E426F15
:10376000436BEF0E446F456BF10E466F476BF20EE5
:10377000486F496BF30E4A6F4B6BF50E4C6F4D6BF8
:10378000F60E4E6F4F6BF70E506F516BF80E526F77
:10379000536BFA0E546F556BFB0E566F576BFC0E46
:1037A000586F596BFE0E5A6F5B6B5C695D6B5E6B9D
:1037B000010E5F6F606F616F030E626F010E636FCA
:1037C000040E646F010E656F050E666F010E676F64
:1037D000060E686F010E696F080E6A6F010E6B6F3F
:1037E000090E6C6F010E6D6F0A0E6E6F010E6F6F1A
:1037F0000C0E706F010E716F0D0E726F010E736FF4
:103800000E0E746F010E756F0F0E766F010E776FCF
:10381000110E786F010E796F120E7A6F010E7B6FA9
:10382000130E7C6F010E7D6F140E7E6F010E7F6F85
:10383000160E806F010E816F170E826F010E836F5F
:10384000180E846F010E856F1A0E866F010E876F3A
:103850001B0E886F010E896F1C0E8A6F010E8B6F15
:103860001D0E8C6F010E8D6F1F0E8E6F010E8F6FF0
:10387000200E906F010E916F210E926F010E936FCB
:10388000230E946F010E956F240E966F010E976FA5
:10389000250E986F010E996F260E9A6F010E9B6F81
:1038A000280E9C6F010E9D6F290E9E6F010E9F6F5B
:1038B0002A0EA06F010EA16F2B0EA26F010EA36F37
:1038C0002D0EA46F010EA56F2E0EA66F010EA76F11
:1038D0002F0EA86F010EA96F310EAA6F010EAB6FEC
:1038E000320EAC6F010EAD6F330EAE6F010EAF6FC7
:1038F000340EB06F010EB16F360EB26F010EB36FA2
:10390000370EB46F010EB56F4C0EB86FB96B4E0E1B
:10391000BA6FBB6B500EBC6FBD6B520EBE6FBF6BF0
:10392000540EC06FC16B560EC26FC36B580EC46F7E
:10393000C56B5A0EC66FC76B5C0EC86FC96B5D0E48
:10394000CA6FCB6B5F0ECC6FCD6B610ECE6FCF6B42
:10395000630ED06FD16B650ED26FD36B670ED46FD1
:10396000D56B690ED66FD76B6B0ED86FD96B6D0E9A
:10397000DA6FDB6B6F0EDC6FDD6B700EDE6FDF6B93
:10398000720EE06FE16B740EE26FE36B760EE46F24
:10399000E56B780EE66FE76B7A0EE86FE96B7C0EED
:1039A000EA6FEB6B7E0EEC6FED6B800EEE6FEF6BE4
:1039B000810EF06FF16B830EF26FF36B850EF46F77
:1039C000F56B870EF66FF76B890EF86FF96B8B0E40
:1039D000FA6FFB6B8D0EFC6FFD6B8F0EFE6FFF6B36
:1039E000910E0D01006F016B930E026F036B940E2D
:1039F000046F056B960E066F076B980E086F096BC8
:103A00009A0E0A6F0B6B9C0E0C6F0D6B9E0E0E6F59
:103A10000F6BA00E106F116BA20E126F136BA40E22
:103A2000146F156BA50E166F176BA70E186F196B19
:103A3000A90E1A6F1B6BAB0E1C6F1D6BAD0E1E6FAC
:103A40001F6BAF0E206F216BB10E226F236BB30E75
:103A5000246F256BB50E266F276BB70E286F296B69
:103A6000B80E2A6F2B6BBA0E2C6F2D6BBC0E2E6FFF
:103A70002F6BBE0E306F316BC00E326F336BC20EC8
:103A8000346F356BC40E366F376BC60E386F396BBB
:103A9000C80E3A6F3B6BCA0E3C6F3D6BCB0E3E6F50
:103AA0003F6BCD0E406F416BCF0E426F436BD10E1B
:103AB000446F456BD30E466F476BD50E486F496B0D
:103AC000D70E4A6F4B6BD90E4C6F4D6BDB0E4E6FA2
:103AD0004F6BDC0E506F516BDE0E526F536BE00E6E
:103AE000546F556BE20E566F576BE40E586F596B5F
:103AF000E60E5A6F5B6BE80E5C6F5D6BEA0E5E6FF5
:103B00005F6BEC0E606F616BEE0E626F636BEF0EBE
:103B1000646F656BF10E666F676BF30E686F696BB0
:103B2000F50E6A6F6B6BF70E6C6F6D6BF90E6E6F47
:103B30006F6BFB0E706F716BFD0E726F736B746940
:103B4000756B766B010E776F020E786F010E796FD1
:103B5000040E7A6F010E7B6F060E7C6F010E7D6F77
:103B6000080E7E6F010E7F6F0A0E806F010E816F4F
:103B70000C0E826F010E836F0E0E846F010E856F27
:103B8000100E866F010E876F120E886F010E896FFF
:103B9000130E8A6F010E8B6F150E8C6F010E8D6FD9
:103BA000170E8E6F010E8F6F190E906F010E916FB1
:103BB0001B0E926F010E936F1D0E946F010E956F89
:103BC0001F0E966F010E976F210E986F010E996F61
:103BD000230E9A6F010E9B6F250E9C6F010E9D6F39
:103BE000260E9E6F010E9F6F280EA06F010EA16F13
:103BF0002A0EA26F010EA36F2C0EA46F010EA56FEB
:103C00002E0EA66F010EA76F300EA86F010EA96FC2
:103C1000320EAA6F010EAB6F340EAC6F010EAD6F9A
:103C2000360EAE6F010EAF6F370EB06F010EB16F73
:103C3000390EB26F010EB36F3B0EB46F010EB56F4C
:063C400000011200FFD795
:020000040030CA
:0300010006170ED1
:020005008580F4
:060008000FC00FE00F40E5
:00000001FF
